:0913300043C80530CEFDE5C922D9
:0713390075CA143004012203
:0E13400043C80530CEFDC2CEE5C930E0EF2235
:07134E0075CA1130040122F1
:0E13550043C80530CEFDC2CEE5C920E0EF2230
:0A13630053C8FB43C80130CEFD2241
:0D136D0075CA0E75C901716375CA1475C982
:03137A000080E60A
:0D137D0075CA0E75C901716375CA1175C975
:03138A000180D609
:04138D00F5C980D24C
:09139100E6F5C9716308D9F822E0
:09139A00E493F5C97163D9F8224E
:0E13A3004386108C828D83EA2CC5F0EB3DA8AA
:0213B100F0F951
:0713B30071397C4075CA216D
:0B13BA007130F0E8B58207E9B583034D
:0313C500716D2225
:0613C800DCF0716D80E510
:0B13CE00714E75CA218C828D83EAF9F4
:0413D900719A717D17
:0313DD00714E222C
:0C13E0008C828D837CF87D001215517406
:0913EC00F5C0E07413C0E0E473E5
:0113F50022D5
:0C13F600438610E4F550F551F552F55314
:0B140200714E75CA217455718D745332
:08140D00718D7442718D74535E
:0C141500718D788479047191789F7904BE
:0614210071917400718D51
:08142700717D714E7904789F7C
:03142F00913222D5
:01143200E4D5
:05143300F608D9FC22BF
:0E14F4007895E6C5F008E6FC08E6FD08E6FA85
:0C15020008E6FBC5F0B4010471A38025CD
:07150E00B4020471E0801E2D
:07151500B4040471CE80173D
:07151C00B41004B138801087
:07152300B41104B16C800952
:07152A00B41204B17080024D
:02153100B151B6
:0515330071F60218181A
:0C153800E4F577F578F579F57A757B7F9E
:08154400757C00757D7F757E4A
:05154C000012128022D4
:05155100B138E4F8F9D7
:0E155600EC120F25ED120F25D3E438F8E4391E
:08156400F9B800EEB940EB22DA
:04156C00B138A18C65
:0E1570008C778D788A798B7A789AE6F57B08ED
:0E157E00E6F57C08E6F57D08E6F57E121280A3
:0A158C007888E6FB08E6FC08E6FD9F
:0E159600EBF5F033CC33CD33FBEC33CD33CB60
:0815A40033FCE5F003541FFDC8
:0B15AC00EB4C601C71397F2075CA21D8
:0C15B7007130120F257130120F25DFF487
:0715C300716D1BBBFF011C51
:0215CA0080E0BF
:0815CC00ED6013713975CA21AD
:0C15D4007130120F257130120F25DDF46C
:0215E000716D2B
:0115E20022E6
:00000001FF
